BL51 BANKED LINKER/LOCATER V5.11                                                        04/23/2014  11:26:56  PAGE 1


BL51 BANKED LINKER/LOCATER V5.11, INVOKED BY:
D:\PROGRAM FILES\KEIL\C51\BIN\BL51.EXE STARTUP.obj, LCD12864.obj TO LCD12864


MEMORY MODEL: SMALL


INPUT MODULES INCLUDED:
  STARTUP.obj (?C_STARTUP)
  LCD12864.obj (LCD12864)


LINK MAP OF MODULE:  LCD12864 (?C_STARTUP)


            TYPE    BASE      LENGTH    RELOCATION   SEGMENT NAME
            -----------------------------------------------------

            * * * * * * *   D A T A   M E M O R Y   * * * * * * *
            REG     0000H     0008H     ABSOLUTE     "REG BANK 0"
            DATA    0008H     0005H     UNIT         _DATA_GROUP_
            IDATA   000DH     0001H     UNIT         ?STACK

            * * * * * * *   C O D E   M E M O R Y   * * * * * * *
            CODE    0000H     0003H     ABSOLUTE     
            CODE    0003H     0140H     UNIT         ?CO?LCD12864
            CODE    0143H     007CH     UNIT         ?PR?MAIN?LCD12864
            CODE    01BFH     004CH     UNIT         ?PR?_HZ_LCDDISP16?LCD12864
            CODE    020BH     0035H     UNIT         ?PR?CLR_SCR?LCD12864
            CODE    0240H     0031H     UNIT         ?PR?_LCDDELAY?LCD12864
            CODE    0271H     002BH     UNIT         ?PR?INIT_LCD?LCD12864
            CODE    029CH     001AH     UNIT         ?PR?CHECKSTATE?LCD12864
            CODE    02B6H     000DH     UNIT         ?PR?_WRITE_COM?LCD12864
            CODE    02C3H     000DH     UNIT         ?PR?_WRITE_DATA?LCD12864
            CODE    02D0H     000CH     UNIT         ?C_C51STARTUP



OVERLAY MAP OF MODULE:   LCD12864 (?C_STARTUP)


SEGMENT                              DATA_GROUP 
  +--> CALLED SEGMENT              START    LENGTH
--------------------------------------------------
?C_C51STARTUP                      -----    -----
  +--> ?PR?MAIN?LCD12864

?PR?MAIN?LCD12864                  -----    -----
  +--> ?PR?INIT_LCD?LCD12864
  +--> ?PR?CLR_SCR?LCD12864
  +--> ?CO?LCD12864
  +--> ?PR?_HZ_LCDDISP16?LCD12864

?PR?INIT_LCD?LCD12864              -----    -----
  +--> ?PR?_LCDDELAY?LCD12864
  +--> ?PR?_WRITE_COM?LCD12864

?PR?_WRITE_COM?LCD12864            -----    -----
BL51 BANKED LINKER/LOCATER V5.11                                                      04/23/2014  11:26:56  PAGE 2


  +--> ?PR?CHECKSTATE?LCD12864
  +--> ?PR?_LCDDELAY?LCD12864

?PR?CHECKSTATE?LCD12864            -----    -----
  +--> ?PR?_LCDDELAY?LCD12864

?PR?CLR_SCR?LCD12864               0008H    0001H
  +--> ?PR?_WRITE_COM?LCD12864
  +--> ?PR?_WRITE_DATA?LCD12864

?PR?_WRITE_DATA?LCD12864           -----    -----
  +--> ?PR?CHECKSTATE?LCD12864
  +--> ?PR?_LCDDELAY?LCD12864

?PR?_HZ_LCDDISP16?LCD12864         0008H    0005H
  +--> ?PR?_WRITE_COM?LCD12864
  +--> ?PR?_WRITE_DATA?LCD12864



SYMBOL TABLE OF MODULE:  LCD12864 (?C_STARTUP)

  VALUE           TYPE          NAME
  ----------------------------------

  -------         MODULE        ?C_STARTUP
  C:02D0H         SEGMENT       ?C_C51STARTUP
  I:000DH         SEGMENT       ?STACK
  C:0000H         PUBLIC        ?C_STARTUP
  D:00E0H         SYMBOL        ACC
  D:00F0H         SYMBOL        B
  D:0083H         SYMBOL        DPH
  D:0082H         SYMBOL        DPL
  N:0000H         SYMBOL        IBPSTACK
  N:0100H         SYMBOL        IBPSTACKTOP
  N:0080H         SYMBOL        IDATALEN
  C:02D3H         SYMBOL        IDATALOOP
  N:0000H         SYMBOL        PBPSTACK
  N:0000H         SYMBOL        PBPSTACKTOP
  N:0000H         SYMBOL        PDATALEN
  N:0000H         SYMBOL        PDATASTART
  N:0000H         SYMBOL        PPAGE
  N:0000H         SYMBOL        PPAGEENABLE
  D:00A0H         SYMBOL        PPAGE_SFR
  D:0081H         SYMBOL        SP
  C:02D0H         SYMBOL        STARTUP1
  N:0000H         SYMBOL        XBPSTACK
  N:0000H         SYMBOL        XBPSTACKTOP
  N:0000H         SYMBOL        XDATALEN
  N:0000H         SYMBOL        XDATASTART
  C:0000H         LINE#         92
  C:02D0H         LINE#         99
  C:02D2H         LINE#         100
  C:02D3H         LINE#         101
  C:02D4H         LINE#         102
  C:02D6H         LINE#         151
  C:02D9H         LINE#         155
BL51 BANKED LINKER/LOCATER V5.11                                                      04/23/2014  11:26:56  PAGE 3


  -------         ENDMOD        ?C_STARTUP

  -------         MODULE        LCD12864
  C:0000H         SYMBOL        _ICE_DUMMY_
  B:00A0H.2       PUBLIC        LCDScs
  D:0080H         PUBLIC        P0
  B:00A0H.4       PUBLIC        LCDDi
  D:00A0H         PUBLIC        P2
  C:02C3H         PUBLIC        _write_data
  C:00A3H         PUBLIC        HZ_cheng
  C:0003H         PUBLIC        HZ_chong
  B:00A0H.6       PUBLIC        LCDEnable
  C:0043H         PUBLIC        HZ_dian
  C:0143H         PUBLIC        main
  C:020BH         PUBLIC        Clr_Scr
  C:02B6H         PUBLIC        _write_com
  C:0083H         PUBLIC        HZ_gong
  C:0023H         PUBLIC        HZ_qing
  C:0123H         PUBLIC        HZ_yuan
  C:0251H         PUBLIC        _LCDdelay
  C:0271H         PUBLIC        init_lcd
  C:00C3H         PUBLIC        HZ_zhi
  C:0103H         PUBLIC        HZ_xue
  C:00E3H         PUBLIC        HZ_ye
  C:029CH         PUBLIC        CheckState
  C:0063H         PUBLIC        HZ_zi
  C:01BFH         PUBLIC        _hz_LCDDisp16
  B:00A0H.1       PUBLIC        LCDMcs
  B:00A0H.5       PUBLIC        LCDRW
  -------         PROC          L?0036
  -------         ENDPROC       L?0036
  -------         PROC          _LCDDELAY
  D:0006H         SYMBOL        t
  -------         DO            
  D:0004H         SYMBOL        i
  D:0006H         SYMBOL        j
  -------         ENDDO         
  C:0251H         LINE#         113
  C:0251H         LINE#         114
  C:0251H         LINE#         116
  C:0262H         LINE#         117
  C:0270H         LINE#         118
  -------         ENDPROC       _LCDDELAY
  -------         PROC          CHECKSTATE
  -------         DO            
  D:0003H         SYMBOL        dat
  D:0003H         SYMBOL        DATA
  -------         ENDDO         
  C:029CH         LINE#         129
  C:029CH         LINE#         130
  C:029CH         LINE#         132
  C:029EH         LINE#         133
  C:02A0H         LINE#         135
  C:02A0H         LINE#         136
  C:02A2H         LINE#         137
  C:02A4H         LINE#         138
  C:02AAH         LINE#         139
BL51 BANKED LINKER/LOCATER V5.11                                                      04/23/2014  11:26:56  PAGE 4


  C:02AAH         LINE#         140
  C:02ACH         LINE#         141
  C:02ACH         LINE#         142
  C:02ACH         LINE#         143
  C:02B5H         LINE#         144
  -------         ENDPROC       CHECKSTATE
  -------         PROC          _WRITE_COM
  D:0002H         SYMBOL        cmdcode
  C:02B6H         LINE#         155
  C:02B8H         LINE#         156
  C:02B8H         LINE#         157
  C:02BBH         LINE#         158
  C:02BDH         LINE#         159
  C:02BDH         LINE#         160
  C:02BDH         LINE#         161
  C:02BDH         LINE#         162
  C:02BDH         LINE#         163
  C:02C0H         LINE#         164
  C:02C2H         LINE#         165
  -------         ENDPROC       _WRITE_COM
  -------         PROC          INIT_LCD
  C:0271H         LINE#         176
  C:0271H         LINE#         177
  C:0271H         LINE#         178
  C:0278H         LINE#         179
  C:027AH         LINE#         180
  C:027CH         LINE#         181
  C:0283H         LINE#         182
  C:0288H         LINE#         183
  C:028DH         LINE#         184
  C:0292H         LINE#         185
  C:0297H         LINE#         186
  -------         ENDPROC       INIT_LCD
  -------         PROC          _WRITE_DATA
  D:0002H         SYMBOL        LCDDispdata
  C:02C3H         LINE#         198
  C:02C5H         LINE#         199
  C:02C5H         LINE#         200
  C:02C8H         LINE#         201
  C:02CAH         LINE#         202
  C:02CAH         LINE#         203
  C:02CAH         LINE#         204
  C:02CAH         LINE#         205
  C:02CAH         LINE#         206
  C:02CDH         LINE#         207
  C:02CFH         LINE#         208
  -------         ENDPROC       _WRITE_DATA
  -------         PROC          CLR_SCR
  -------         DO            
  D:0001H         SYMBOL        j
  D:0008H         SYMBOL        k
  -------         ENDDO         
  C:020BH         LINE#         219
  C:020BH         LINE#         220
  C:020BH         LINE#         222
  C:020DH         LINE#         223
  C:020FH         LINE#         224
BL51 BANKED LINKER/LOCATER V5.11                                                      04/23/2014  11:26:56  PAGE 5


  C:0214H         LINE#         225
  C:0219H         LINE#         226
  C:021CH         LINE#         227
  C:021CH         LINE#         228
  C:0224H         LINE#         229
  C:0226H         LINE#         230
  C:0226H         LINE#         231
  C:022DH         LINE#         232
  C:0232H         LINE#         233
  C:0236H         LINE#         234
  C:023FH         LINE#         235
  -------         ENDPROC       CLR_SCR
  -------         PROC          _HZ_LCDDISP16
  D:0008H         SYMBOL        page
  D:0009H         SYMBOL        column
  D:000AH         SYMBOL        hzk
  -------         DO            
  D:0001H         SYMBOL        j
  D:000CH         SYMBOL        i
  -------         ENDDO         
  C:01BFH         LINE#         246
  C:01C7H         LINE#         247
  C:01C7H         LINE#         248
  C:01CBH         LINE#         249
  C:01CBH         LINE#         250
  C:01CBH         LINE#         251
  C:01D4H         LINE#         252
  C:01DCH         LINE#         253
  C:01DFH         LINE#         254
  C:0206H         LINE#         255
  C:020AH         LINE#         256
  -------         ENDPROC       _HZ_LCDDISP16
  -------         PROC          MAIN
  C:0143H         LINE#         267
  C:0143H         LINE#         268
  C:0143H         LINE#         269
  C:0146H         LINE#         270
  C:0149H         LINE#         271
  C:014BH         LINE#         272
  C:014DH         LINE#         273
  C:0157H         LINE#         274
  C:0162H         LINE#         275
  C:016DH         LINE#         276
  C:0178H         LINE#         277
  C:0183H         LINE#         278
  C:0185H         LINE#         279
  C:0187H         LINE#         280
  C:0191H         LINE#         281
  C:019CH         LINE#         282
  C:01A7H         LINE#         283
  C:01B2H         LINE#         284
  C:01BDH         LINE#         285
  C:01BDH         LINE#         286
  C:01BDH         LINE#         288
  -------         ENDPROC       MAIN
  -------         ENDMOD        LCD12864

BL51 BANKED LINKER/LOCATER V5.11                                                      04/23/2014  11:26:56  PAGE 6


Program Size: data=14.0 xdata=0 code=732
LINK/LOCATE RUN COMPLETE.  0 WARNING(S),  0 ERROR(S)
